:0E0000000C9459000C9400000C9400000C9419
:10000E0000000C9400000C948C000C94A3000C9433
:10001E00BE000C9400000C9400000C9400000C9494
:10002E0000000C9400000C9400000C9400000C9442
:10003E0000000C9400000C9400000C9400000C9432
:10004E0000000C9400000C9400000C9400000C9422
:10005E0000000C9400000C9400000C9400000C9412
:10006E0000000C9400000C9400000C9400000C9402
:10007E0000000C9400000C9400000C94000002028E
:10008E000024743E01002D4E414E00494E460000A4
:10009E0002000C008C000400BC068E000100C90694
:1000AE0092000000F894EE27ECBBF1E0F5BFE5BF3F
:1000BE00E0936C00F8E1F1BDE1BD8DE0A2E0BB275D
:1000CE00ED938A95E9F780E090E1A0E0B1E0ED9341
:1000DE000197E9F7EEE9F0E085919591009761F0CF
:1000EE00A591B59105901590BF01F00105900D9267
:1000FE000197E1F7FB01F0CF8BBFEFEFEDBFE0E132
:10010E00EEBFC0E0D5E00C947409FA92EA93EFB713
:10011E00EA93E8940D996894F0F8F0FC05C0839486
:10012E00E8E08E1608F08824F0FE05C0882011F451
:10013E00E8E08E2E8A9416C0FA92EA93EFB7EA930D
:10014E00E8940C996894F0F8F0FC05C08394E8E00C
:10015E008E1608F08824F0FE05C0882011F4E8E021
:10016E008E2E8A94E991EFBFE991F9901895AA9392
:10017E00EA93FA93EFB7EA93E82DF0E0309711F493
:10018E00E8E05FC0E130A0E0FA0711F4E9E059C001
:10019E00E230A0E0FA0711F4EAE053C0E330A0E049
:1001AE00FA0711F4EBE04DC0E430A0E0FA0711F4C9
:1001BE00ECE047C0E530A0E0FA0711F4EDE041C0F5
:1001CE00E630A0E0FA0711F4EEE03BC0E730A0E025
:1001DE00FA0711F4EFE035C0E830A0E0FA0711F4A9
:1001EE00882430C0E930A0E0FA0711F4E1E029C01C
:1001FE00EA30A0E0FA0721F1EB30A0E0FA0711F4A3
:10020E00E3E01FC0EC30A0E0FA0711F4E4E019C0FF
:10021E00ED30A0E0FA0711F4E5E013C0EE30A0E0F7
:10022E00FA0711F4E6E00DC0EF30A0E0FA0711F482
:10023E00E0E107C0E031A0E0FA0711F4E7E001C009
:10024E00E2E08E2EE991EFBFF991E991A99118950F
:10025E00AA93E0919B00E072E1F3E881E0939C00A9
:10026E0010C00E94C60AA9810E943F0FA8810E9459
:10027E003F0F82C10E94C60AA8810E943F0F0E94B2
:10028E001A0F219608950E94C60AE981E06CAE2FDE
:10029E000E943F0FA881AF3228F40E94CC0AA0E042
:1002AE000E943F0FA881AF3219F4A8E00E94D20A33
:1002BE00A881A03319F4AFE30E94D50AA881A13317
:1002CE0031F4A6E00E943F0FA2E00E94DD0AA88151
:1002DE00A23319F4ABE50E94E20AA881A33319F404
:1002EE00AFE40E94E20AA881A43319F4A6E60E94A4
:1002FE00E20AA881A53319F4ADE60E94E20AA881AC
:10030E00A63319F4ADE70E94E20AA881A73319F4C7
:10031E00A7E00E94D20AA881A83319F4AFE70E9481
:10032E00E20AA881A93319F4AFE60E94E20AA88175
:10033E00AA3331F4A0E00E943F0FA0E40E94DD0A30
:10034E00A881AB3331F4A0E00E943F0FA0E90E94D8
:10035E00DD0AA881AC3331F4A0E40E943F0FA5ED75
:10036E000E94DD0AA881AD3319F4A0E40E94E20ACE
:10037E00A881AE3331F4A0EC0E943F0FAFEF0E9484
:10038E00DD0AA881AF3319F4A0E00E94D50AA88136
:10039E00A03431F4A0E00E943F0FA0E10E94DD0ADC
:1003AE00A881A13419F4A7E70E94E20AA881A23419
:1003BE0031F4A9E70E943F0FAAE80E94DD0AA88146
:1003CE00A33419F4A9E30E94D20AA881A43419F423
:1003DE00AFE30E94D20AA881A53431F4A9E70E94A6
:1003EE003F0FA0E80E94DD0AA881A63419F4A1E708
:1003FE000E94E20AA881A73431F4ADE30E943F0FB8
:10040E00A4E00E94DD0AA881A83419F4A6E70E9490
:10041E00E20AA881A93431F4A9E00E943F0FA1EDB0
:10042E000E94DD0AA881AA3419F4AEE00E94D20A15
:10043E00A881AB3431F4A0E70E943F0FAAE80E94D6
:10044E00DD0AA881AC3419F4A8E30E94D20AA8816F
:10045E00AD3431F4A6EB0E943F0FA2EC0E94DD0AF0
:10046E00A881AE3431F4A6EB0E943F0FA8E80E949B
:10047E00DD0AA881AF3419F4AFE30E94D20AA88135
:10048E00A03519F4A3E70E94E20AA881A13531F440
:10049E00AFE30E943F0FA8E00E94DD0AA881A235BB
:1004AE0031F4A3E70E943F0FACE80E94DD0AA88159
:1004BE00A33519F4ADE60E94E20AA881A43531F401
:1004CE00A1E00E943F0FA1ED0E94DD0AA881A53593
:1004DE0019F4AEE30E94D20AA881A63531F4A0E841
:1004EE000E943F0FA2E90E94DD0AA881A73531F4D0
:1004FE00A6E30E943F0FA8EA0E94DD0AA881A83554
:10050E0031F4A0E80E943F0FAAEA0E94DD0AA881FA
:10051E00A93531F4A2E60E943F0FA4E90E94DD0A3C
:10052E00A881AA3519F4A9E00E94D50AA881AB3595
:10053E0019F4A9E30E94D20AA881AC3531F4A0E8DF
:10054E000E943F0FA8E80E94DD0AA881AD3519F47C
:10055E00AFE00E94D20AA881AE3531F4AFEF0E940F
:10056E003F0FAFEF0E94DD0AA881AF3528F00E9441
:10057E00CC0AA0E00E943F0F0E941A0F2296089507
:10058E005524ECE05E1630F40E94E60AA3E67BDE0C
:10059E005394F7CF08955524ECE05E1630F40E9484
:1005AE00E60AAEE570DE5394F7CF0895E6E0EA93DF
:1005BE00ADE403C0E6E0EA93ABE465DEE3E0EA9384
:1005CE00A8E40E94EF0AAAE55EDE0895AA931A93A4
:1005DE00A981A33079F414E8EA811E1710F014569D
:1005EE00FBCFEA81E11BEA83A12FB0E0E4E6F0E065
:1005FE000E94F40AA981A23079F41AE5EA811E1745
:10060E0010F01A50FBCFEA81E11BEA83A12FB0E074
:10061E00EAE0F0E00E94F40AA981A13071F419E039
:10062E00EA811E1710F01150FBCFEA81E11BEA831D
:10063E00EB81EA93A12FA05D26DE18812496089502
:10064E000E94040B0E943A0B0F9B03C0E0E0E815DA
:10065E0009F004C083E08A95F1F7F6CF0E94420BB1
:10066E000F9906C00E944C0B81E28A95F1F7F8CFE4
:10067E000E94570BA732E2E0BE07E0E08E07E0E0F3
:10068E009E0750F00E94570BAA38E2E0BE07E0E04A
:10069E008E07E0E09E0708F0C2C00E94420B0F9B3F
:1006AE0009C00E944C0B31976040704081E28A95E0
:1006BE00F1F7F5CF0E94570BA431E1E0BE07E0E061
:1006CE008E07E0E09E0750F00E94570BA534E1E044
:1006DE00BE07E0E08E07E0E09E0708F01FC055243D
:1006EE000E94420B0F9904C081E18A95F1F7FACF6F
:1006FE000F9B09C00E944C0B31976040704081E106
:10070E008A95F1F7F5CF0E94600BA0910005A083AA
:10071E0053940E94420BE0E25E1620F30E94650B9A
:10072E005524E0E25E1680F40E94600B9080EEE6A7
:10073E009E1620F40E94600BA0E003C00E94600B86
:10074E00A1E0A0835394EDCF5524E8E05E1630F57A
:10075E000E946A0B7E2F8F2F0E946F0BEC5FFA4F59
:10076E0060810E946F0BEB5FFA4FE081EE0F6E0F10
:10077E000E946F0BEA5FFA4FE081EE0FEE0F6E0FE5
:10078E000E946F0BE95FFA4FE081EE0FEE0FEE0F56
:10079E00E60FA72FB82FEC935394D7CFF1DEE1E2FB
:1007AE000E94740BEEE10E94780BEBE10E947C0B31
:1007BE00E8E10E94800B5524E8E05E1608F5E52D71
:1007CE00A3E0EA02F001A5E1AE1B9A2E0E946A0B8D
:1007DE00A081AA3038F49A920E946A0BE081E05D03
:1007EE00AE2F51DD0E946A0BA081AA3038F09A928A
:1007FE000E946A0BE081E95CAE2F45DD5394DCCF9D
:10080E005524E8E05E1630F40E946A0BA08120DDCC
:10081E005394F7CFE1E4EA93A6E00E94840B089587
:10082E000E94040B0E943A0B0F9B03C0E1E0E815F7
:10083E0009F004C083E08A95F1F7F6CFE5E05E2E6D
:10084E00E1E0E0930405E0930505E0930605E093EF
:10085E000705E0930805A52DB0E0AC5FBA4FE0E0C8
:10086E000F99E1E0EC930E948A0B5394EFEF5E1622
:10087E0090F30E94650B772466244424E72DF0E064
:10088E00EC5FFA4F0080A72DBB27E42DF0E0EA0FB6
:10089E00FB1FEC5FFA4FE081E01511F44394EECFAD
:1008AE00E62DF0E0EC5FF94F4082740C4424639423
:1008BE00EFEF7E1618F355244424E0E24E1668F549
:1008CE000E948F0B28F40E94600BA1E0A08353942A
:1008DE000E948F0B50F00E94600BA1E0A0835394F6
:1008EE000E94600BA1E0A083539443940E948F0B4F
:1008FE0028F40E94600BA0E0A08353940E948F0BFB
:10090E0050F00E94600BA0E0A08353940E94600BF5
:10091E00A0E0A08353944394D0CF55244424E0E226
:10092E004E1650F5E42DF0E0EC5FFA4FA081A130A9
:10093E0039F4E42DF0E0EB5FFA4FA081A03009F01E
:10094E0004C00E946A0BA1E0A083E42DF0E0EC5FEE
:10095E00FA4FA081A03039F4E42DF0E0EB5FFA4FAE
:10096E00A081A13009F004C00E946A0BA0E0A08310
:10097E00439443945394D3CF03DEE1E20E94960B4B
:10098E00EEE10E947C0BEBE1EA93A5E37CDCE8E16F
:10099E000E94800BA0918606A13021F4E5E1EA9336
:1009AE00A1E371DCE0918606E03019F4E5E10E94E6
:1009BE009A0BE2E10E949E0BE0918806EE0FEE0F7D
:1009CE00EE0FAE2FE0918906EE0FEE0FAE0FE09117
:1009DE008A06EE0FAE0FE0918B06EA0F9E2EEFE029
:1009EE00EA939A92A2E0F2DDE9E00E949E0BE0917A
:1009FE008506A0E4EA02602DE0918C06A0E2EA02F0
:100A0E00F0016E0FE0918D06A0E1EA02F001A62F33
:100A1E00AE0FE0918E06EE0FEE0FEE0FAE0FE091E1
:100A2E008F06EE0FEE0FAE0FE0919006EE0FAE0FAB
:100A3E00E0919106EA0F9E2EE6E0EA939A92A3E0E9
:100A4E00C5DDE1E4EA93A6E00CDCE1E0E81521F473
:100A5E00A0EDB7E00E94570F0895E1E2EA93A9E3F3
:100A6E000E94A20BA6E30FDCEBE10E949A0BE8E1D9
:100A7E000E949A0BE5E10E94A70BE2E1EA93A8E33C
:100A8E0002DCEFE00E94A70BECE00E94740BE9E0A1
:100A9E000E94A70BE6E0EA93A1E30E94AB0BAFE541
:100AAE000E94EF0AAFE5EFDBE4E0E81509F04DC078
:100ABE00A3E40E94B00BA4E5CBDBA8E4C9DBADE256
:100ACE00C7DBA6E3C5DBA0E30E94B50BA2E40E9440
:100ADE00B50BA6E4BDDBA2E50E94B00BA1E5B8DB29
:100AEE00A5E50E94B00BAEE4B3DBA3E4B1DBA9E550
:100AFE000E94B50BA3E4ACDBAFE4AADBA5E5A8DB53
:100B0E00AEE4A6DBA4E50E94B00BA2E50E94B50BF5
:100B1E00A2E50E94B00BA6E59BDBAEE20E94B50BF0
:100B2E00A1E396DBAEE294DBA1E392DBA0E390DBE4
:100B3E00ADE08EDBAAE00E94B50BE4E0E81521F4EF
:100B4E00A7EEB3E00E94570FAFCF08950E94BA0BE5
:100B5E000E94C10BE5E10E947C0B0E94C80BE9E0EC
:100B6E000E94800BE6E00E94740BE3E0EA93A5E49A
:100B7E000E94EF0AA3E487DB882019F40E948A0BF7
:100B8E00FBCF08950E94BA0B0E94C10BE5E10E94B3
:100B9E007C0B0E94C80BE9E00E94800BE6E00E94ED
:100BAE00960BE3E0EA93A3E40E94EF0AA5E36BDB66
:100BBE00E1E0E81519F40E948A0BFACF0895E1E2FC
:100BCE00EA93A6E40E94A20BA5E50E94D40BA4E52D
:100BDE000E94D90BA5E557DBE5E10E94960BE2E1F9
:100BEE000E94780BEFE00E94800B0E94DE0BA3E5C3
:100BFE004ADBE6E00E94780BE3E0EA93AFE50E9461
:100C0E00EF0AAFE540DBE7E0E81519F40E948A0B26
:100C1E00FACFEFE0E81519F40E948A0BFACFE0E163
:100C2E00E81519F40E948A0BFACF0895E1E2EA93CF
:100C3E00A5E50E94A20BA1E426DBEBE10E94960B38
:100C4E00E8E10E94E60BE5E10E94800BE2E10E94E2
:100C5E00E60BEFE00E94780BECE0EA93A3E513DBE2
:100C6E00E9E00E94E60BE6E00E94800BE3E0EA93E7
:100C7E00AFE50E94EF0AAFE506DBE6E0E81519F4F2
:100C8E000E948A0BFACF08950E94EA0BEBE10E94B4
:100C9E00780B0E94F10BEFE00E94740BECE00E94C7
:100CAE007C0B0E94FD0BE3E0EA93A1E40E94EF0AA5
:100CBE00AFE5E9DAE2E0E81519F40E948A0BFACF03
:100CCE0008950E94EA0BEBE10E94780B0E94F10B53
:100CDE00EFE00E94740BECE00E947C0B0E94FD0B77
:100CEE00E3E0EA93A2E40E94EF0AAFE5CCDAE3E098
:100CFE00E81519F40E948A0BFACF08950E94EA0BA8
:100D0E00EBE10E94780B0E94040C0E949E0B0E9445
:100D1E001A0CAEE20E94EF0AAEE2B5DAE4E0E81594
:100D2E0019F40E948A0BFACF08950E94EA0BEBE1A8
:100D3E000E94780B0E94040CEA93AFE3A4DA0E949F
:100D4E001A0CAEE20E94EF0AAEE29DDAE5E0E8157B
:100D5E0019F40E948A0BFACF0895E1E20E94780BF3
:100D6E00EEE10E94960BEBE10E94960BE8E1EA930E
:100D7E00AFE489DAE5E10E94960BE2E10E94230CD2
:100D8E00EFE00E94230CECE00E94230CE9E00E94AD
:100D9E00230CE6E0EA93AEE20E94AB0BAEE20E94B9
:100DAE00EF0AAEE270DAE3E6E81519F40E948A0B58
:100DBE00FACF08951A931A9A1B9A0E94270C0E9432
:100DCE002C0C21F483E08A95F1F7F9CFB09B0CC07F
:100DDE000E94370C0E949A0C0E94B10C0E94BA0C11
:100DEE000E94CD0C0E94D60CB0990AC00E94F20C43
:100DFE000E94550D0E946C0D0E94750D0E94880D6B
:100E0E00B09B02C00E94A50DB09902C00E94650B56
:100E1E00E0E3E093AC060E94AA0D0E94B30D18F019
:100E2E000E94BB0DF8CFE0E3E093AD060E94D50D16
:100E3E0018F00E94DE0DFACFE0E3E093AE060E94BA
:100E4E00F80D18F00E94010EFACFE0E3E093AF0622
:100E5E000E941B0E18F00E94240EFACFE0E3E093DE
:100E6E00B0060E943E0E18F00E94470EFACFE0E345
:100E7E00E093B1060E94610E18F00E946A0EFACF3E
:100E8E00E0E3E093B2060E94840E18F00E948D0EED
:100E9E00FACFA091AC06A03319F4E0E2E093AC06D1
:100EAE00A091AD06A03321F4A091AC06A03209F0BA
:100EBE0003C0E0E2E093AD06A091AE06A03321F4AC
:100ECE00A091AD06A03209F003C0E0E2E093AE06B9
:100EDE00A091AF06A03321F4A091AE06A03209F086
:100EEE0003C0E0E2E093AF06A091AD06A03368F434
:100EFE000E94A70E0E94AC0E0E94AF0E0E94B20E70
:100F0E000E94B60E0E94BE0E55DBA091AD06A03318
:100F1E0048F00E94A70E0E94CF0E0E94D50E0E948E
:100F2E00DE0E44DBD8C11A931A981B980E94270C28
:100F3E000E942C0C21F483E08A95F1F7F9CFB09B37
:100F4E000CC00E94370C0E949A0C0E94B10C0E9499
:100F5E00BA0C0E94CD0C0E94D60CB0990AC00E9409
:100F6E00F20C0E94550D0E946C0D0E94750D0E9490
:100F7E00880DB09B02C00E94A50DB09902C00E94C0
:100F8E00650BE0E3E093AC060E94AA0D0E94B30D40
:100F9E0018F00E94BB0DF8CFE0E3E093AD060E947F
:100FAE00D50D18F00E94DE0DFACFE0E3E093AE0609
:100FBE000E94F80D18F00E94010EFACFE0E3E093C4
:100FCE00AF060E941B0E18F00E94240EFACFE0E32B
:100FDE00E093B0060E943E0E18F00E94470EFACF24
:100FEE00E0E3E093B1060E94610E18F00E946A0ED3
:100FFE00FACFE0E3E093B2060E94840E18F00E944E
:10100E008D0EFACFA091AC06A03319F4E0E2E09376
:10101E00AC06A091AD06A03321F4A091AC06A0328F
:10102E0009F003C0E0E2E093AD06A091AE06A03356
:10103E0021F4A091AD06A03209F003C0E0E2E093E6
:10104E00AE06A091AF06A03321F4A091AE06A03259
:10105E0009F003C0E0E2E093AF06A091AD06A03325
:10106E0068F40E94A70E0E94AC0E0E94AF0E0E9462
:10107E00B20E0E94B60E0E94BE0E9CDAA091AD0674
:10108E00A03348F00E94A70E0E94CF0E0E94D50EEC
:10109E000E94DE0E8BDA1FC11A931A9A1B980E94B9
:1010AE00270C0E942C0C21F483E08A95F1F7F9CFDE
:1010BE00B09B1FC00E94370C0E949A0C0E94B10C6C
:1010CE000E94BA0C0E94CD0C0E94B10C0E94E50E3B
:1010DE00ED2D0E94EC0EE093C006F093C1066093D6
:1010EE00C2067093C3069798A1E0B0E00E94570F16
:1010FE00979AB0991FC00E94F20C0E94550D0E9443
:10110E006C0D0E94750D0E94CD0C0E946C0D0E94FC
:10111E00E50EEC2D0E94EC0EE093C406F093C5068E
:10112E006093C6067093C7069598A1E0B0E00E9442
:10113E00570F959AB09B02C00E94A50DB09902C0A0
:10114E000E94650B0E94F40E0E94FD0E0E94FA0F83
:10115E00DF01CB010E94760ADF01CB010E94AF0AAC
:10116E00A8EBB6E00E948E0F0E940711EEE2E0930C
:10117E00C8060E94FD0E0E94F40E0E949A1009F0FD
:10118E0008F403C0EDE3E093C806E091C006F091C9
:10119E00C1066091C2067091C306A091C406B091BB
:1011AE00C5068091C6069091C7060E949A1009F056
:1011BE0008F403C0ECE3E093C806E0E3E093AC066A
:1011CE000E94AA0D0E94B30D18F00E94BB0DF8CF1D
:1011DE00E0E3E093AD060E94D50D18F00E94DE0DFF
:1011EE00FACFE0E3E093AE060E94F80D18F00E94ED
:1011FE00010EFACFE0E3E093AF060E941B0E18F04B
:10120E000E94240EFACFE0E3E093B0060E943E0E59
:10121E0018F00E94470EFACFE0E3E093B1060E9469
:10122E00610E18F00E946A0EFACFE0E3E093B20668
:10123E000E94840E18F00E948D0EFACFA091AC067B
:10124E00A03319F4E0E2E093AC06A091AD06A03312
:10125E0021F4A091AC06A03209F003C0E0E2E093C5
:10126E00AD06A091AE06A03321F4A091AD06A0323A
:10127E0009F003C0E0E2E093AE06A091AF06A03302
:10128E0021F4A091AE06A03209F003C0E0E2E09393
:10129E00AF06A091AD06A03388F4E1E2EA93A091E7
:1012AE00C8060E94A20B0E94AC0E0E94AF0E0E94B6
:1012BE00B20E0E94B60E0E94BE0E7CD9A091AD0653
:1012CE00A03348F00E94A70E0E94CF0E0E94D50EAA
:1012DE000E94DE0E6BD919910895EFEFEABBE0E0A4
:1012EE00EBBBECEFE7BBE0E0E8BBE4BBE5BBE0EF5C
:1012FE00E1BBE0E0E2BBECE0E2B9E0E0E3B9E093B1
:10130E006100E0936200E0936400E0936500E0BF4B
:10131E00E3BFE2BFE1BFEFBDEEBDEDBDECBDE7BD8E
:10132E00E6BDEBBDEABDE9BDE8BDE0937900E09313
:10133E007800E5BDE4BDE3BDE0938B00E0938A0049
:10134E00E0938900E0938800E0938100E0938000B1
:10135E00E0938700E0938600E0938500E09384009D
:10136E00E0938300E0938200E7BFE0937D00E0937B
:10137E006A00EEE2EABFE0E7E9BFE8BFE0E0EAB903
:10138E00E0939B00E8E0E0939A00E6E0E0939D0096
:10139E00E0E0E0939800E0E4E0939900E0E8E8B93B
:1013AE00E0E0E0BDE6B9EDB9E09374000E94060FEF
:1013BE00AFE90E9441017894E3D8EEE10E947C0BE4
:1013CE00EBE1EA93A8E40E94D90BA1E40E944A0142
:1013DE00E5E10E94740BE2E1EA93A7E40E944A0160
:1013EE00EFE0EA93A0E50E944A010E94DE0BA1E421
:1013FE000E944A01E6E0EA93ABE40E944A01E1E46E
:10140E00EA93A7E00E94840BC6D8A0EDB7E00E9435
:10141E00570FB6D8ECE08E2EE82DF0E0309711F491
:10142E0095DB5BC0E830A0E0FA0711F409D955C08E
:10143E00E130A0E0FA0711F4A5DB4FC0E930A0E0DF
:10144E00FA0711F4EDD949C0E230A0E0FA0711F421
:10145E001BDC43C0EA30A0E0FA0711F4ABDC3DC060
:10146E00E330A0E0FA0711F42CDC37C0EB30A0E03B
:10147E00FA0711F458DD31C0E430A0E0FA0711F498
:10148E003DDC2BC0EC30A0E0FA0711F405DE25C0E0
:10149E00E530A0E0FA0711F448DC1FC0E630A0E00A
:1014AE00FA0711F4C3DB19C0EE30A0E0FA0711F40D
:1014BE00D4DA13C0E730A0E0FA0711F480DB0DC0D8
:1014CE00EF30A0E0FA0711F47ADB07C0E031A0E0BC
:1014DE00FA0711F474DB01C040DC9ECFFFCF0E94EF
:1014EE002011E991F991699179917F7708950E9480
:1014FE0020117B816A81F981E88177FB770F67FD87
:10150E007160972F9E5781F078F0983190F4AA274A
:10151E00BB27882708948795B795A7959A95D1F7F5
:10152E00EA23FB23682305C0E8947727EE27FF27DD
:10153E0066276F77769508F4606877F9A991B99167
:10154E0089919991EA17FB076807790797FB089528
:10155E000E9420110E9416110E947E0A0E941B11E9
:10156E0019F40E94111109C0E6F70E941111A0E0B2
:10157E00B0E080E89FE30E94FA0F24960895AA93A4
:10158E000E940B0FAEEA0C943F0FA0E00E943F0F9B
:10159E00A0E00C943F0F0E943F0FF7CF0E943F0F29
:1015AE00A2EA0E943F0FA0E00C943F0F0E943F0F53
:1015BE00A0E00C943F0F0E943F0FA4E8F7CFE52D5B
:1015CE00A3E0EA02F001A1E2AE1B4A2E4A92089570
:1015DE000E944A01E0E0EA9308950E94EF101E2F48
:1015EE00EB81EA93A12FA05D0E944A01EB81E350AB
:1015FE00EB83E981E150E9830895E1E2EA93A0E506
:10160E000E944A01EEE1EA93A2E50E944A01EBE153
:10161E00EA93A5E40E944A01E8E1EA93A3E50E9459
:10162E004A01E5E1EA93A3E50E944A01E2E1EA9369
:10163E00AFE50E944A01EFE0EA93ABE40E944A0153
:10164E00ECE0EA93A5E40E944A01E9E0EA93A9E5F9
:10165E000E944A01E6E0EA93AFE50E944A01E3E008
:10166E00EA93AFE5B5CFAFE50E944A01E1E4EA9314
:10167E00A6E00C943801E0E0E0930005E09301054C
:10168E00E0930205E09303050895A0E0B5E00E9403
:10169E000211EF5FFF4F6F4F7F4F0E940C110895A5
:1016AE00A0910005B091010580910205909103056E
:1016BE000895E52DF0E0EC5FFA4F0895E1E4EA932A
:1016CE00A5E00C943801E52DF0E0EC57F94F0895A4
:1016DE00A52DE4E0EA9FF0010895EA93AEE40C94A0
:1016EE004A01EA93A5E40C944A01EA93A3E40C940C
:1016FE004A01EA93AFE50C944A010E943801A0ED2D
:10170E00B7E00C94570F8AEF90E00197F1F7089528
:10171E00E42DF0E0EC5FF94FA081AF300895EA932D
:10172E00A2E50C944A01EA93A0E30C944A01EA93D1
:10173E00ADE30C944A010E944A01EEE1EA9308954A
:10174E00EA93A0E40C944A010E944A01E3E0EA9372
:10175E0008950E942F01A5E40C942F010E942F01E1
:10176E00A0E20C942F01E1E2EA93A9E40E944A015F
:10177E00EEE1D5CFEBE1EA93A4E40E944A01E8E161
:10178E00B0CFE2E1EA93AFE40E944A01EFE0EA93C0
:10179E00A4E40E944A01ECE0A4CF0E944A01EBE1CE
:1017AE00EA9308950E944A01E8E1EA930895ECE075
:1017BE00EA93A5E50E944A01E9E0EA930895EA93C7
:1017CE00A4E50C944A01E1E2EA93A6E40E944A01E0
:1017DE00EEE1A5CFE8E1EA93A1E50E944A01E5E139
:1017EE00EA93A5E50E944A01E2E17BCFE9E0EA93A4
:1017FE00A9E50E944A01E6E07CCFE8E1EA93A1E583
:10180E000E944A01E5E1EA93AEE20E944A01E2E15A
:10181E00EA93A2E40E944A01EFE0EA93AEE20E944C
:10182E004A01ECE00895E9E0EA93AEE20E944A0133
:10183E00E6E0EA93A1E488CFEA93AEE20C944A0183
:10184E00E0E0B099E1E01E2F0895E0E0B099E1E00C
:10185E00A12FB0E0F0E0E7FDFFEFEA17FB070895D8
:10186E00969AA1E0B0E00E94570F9698DD9ADC9A06
:10187E00DB9AA1E0B0E00E94570FE3B3FF27662783
:10188E007727E093A406F093A5066093A6067093BF
:10189E00A706A091A406B091A5068091A6069091E8
:1018AE00A706E8E00E94CB10E093A406F093A506ED
:1018BE006093A6067093A706DD9ADC9ADB98A1E0EA
:1018CE00B0E00E94570FE3B3A091A406B091A50615
:1018DE008091A6069091A706FF27662777270E947C
:1018EE00BA10E093A406F093A5066093A606709333
:1018FE00A706A091A406B091A5068091A606909188
:10190E00A706E8E00E94CB10E093A406F093A5068C
:10191E006093A6067093A706DD9ADC98DB9AA1E089
:10192E00B0E00C94570FE3B3A091A406B091A506B6
:10193E008091A6069091A706FF27662777270E941B
:10194E00BA10E093A406F093A5066093A6067093D2
:10195E00A7060895A091A406B091A5068091A606AB
:10196E009091A7060895E8E00E94CB10E093A4069C
:10197E00F093A5066093A6067093A706DD9ADC98F1
:10198E00DB98A1E0B0E00E94570FCDCFE091BC06EE
:10199E00F091BD066091BE067091BF060895DADF24
:1019AE000E9425110E944C10DF01CB01ED2DF0E0BD
:1019BE000E94D7100E94C70F0E944C10A8EBB6E0F1
:1019CE000E948E0F0E9407119798A1E0B0E00E942E
:1019DE00570F979A0895949AA1E0B0E00E94570F7E
:1019EE009498DD98DC9ADB9AA1E0B0E00E94570F44
:1019FE00E3B3FF2766277727E093A806F093A9069F
:101A0E006093AA067093AB06A091A806B091A906A2
:101A1E008091AA069091AB06E8E00E94CB10E0936D
:101A2E00A806F093A9066093AA067093AB06DD98FC
:101A3E00DC9ADB98A1E0B0E00E94570FE3B3A091CF
:101A4E00A806B091A9068091AA069091AB06FF2731
:101A5E00662777270E94BA10E093A806F093A9068E
:101A6E006093AA067093AB06A091A806B091A90642
:101A7E008091AA069091AB06E8E00E94CB10E0930D
:101A8E00A806F093A9066093AA067093AB06DD989C
:101A9E00DC98DB9AA1E0B0E00C94570FE3B3A09171
:101AAE00A806B091A9068091AA069091AB06FF27D1
:101ABE00662777270E94BA10E093A806F093A9062E
:101ACE006093AA067093AB060895A091A806B091F4
:101ADE00A9068091AA069091AB060895E8E00E94AF
:101AEE00CB10E093A806F093A9066093AA06709314
:101AFE00AB06DD98DC98DB98A1E0B0E00E94570FB2
:101B0E00CDCF44DFE2DF0E9425110E944C10DF0191
:101B1E00CB01EC2DF0E00E94D7100E94C70F0E945F
:101B2E004C10A8EBB6E00E948E0F0E9407119598FC
:101B3E00A1E0B0E00E94570F959A0895E1E4EA9370
:101B4E00A3E00C943801A091B806B091B90680912B
:101B5E00BA069091BB060895A034E2E4BE07EFE00A
:101B6E008E07E0E09E070895E091AC06EF5FE093EC
:101B7E00AC06E091B806F091B9066091BA06709184
:101B8E00BB06E054F2446F407040E093B806F09309
:101B9E00B9066093BA067093BB060895D4DFA03AD7
:101BAE00E6E8BE07E1E08E07E0E09E070895E091CB
:101BBE00AD06EF5FE093AD06E091B806F091B90681
:101BCE006091BA067091BB06E05AF64861407040CB
:101BDE00E093B806F093B9066093BA067093BB060D
:101BEE000895B1DFA031E7E2BE07E0E08E07E0E046
:101BFE009E070895E091AE06EF5FE093AE06E0918A
:101C0E00B806F091B9066091BA067091BB06E05124
:101C1E00F74260407040E093B806F093B9066093C7
:101C2E00BA067093BB0608958EDFA83EE3E0BE07AA
:101C3E00E0E08E07E0E09E070895E091AF06EF5FCB
:101C4E00E093AF06E091B806F091B9066091BA063E
:101C5E007091BB06E85EF34060407040E093B806BA
:101C6E00F093B9066093BA067093BB0608956BDFC6
:101C7E00A436E0E0BE07E0E08E07E0E09E070895A0
:101C8E00E091B006EF5FE093B006E091B806F091F8
:101C9E00B9066091BA067091BB06E456F0406040FA
:101CAE007040E093B806F093B9066093BA0670934D
:101CBE00BB06089548DFAA30E0E0BE07E0E08E07DD
:101CCE00E0E09E070895E091B106EF5FE093B10664
:101CDE00E091B806F091B9066091BA067091BB0614
:101CEE00EA50F04060407040E093B806F093B906B9
:101CFE006093BA067093BB06089525DFA130E0E02D
:101D0E00BE07E0E08E07E0E09E070895E091B20680
:101D1E00EF5FE093B206E091B806F091B9066091DC
:101D2E00BA067091BB06E150F04060407040E093FF
:101D3E00B806F093B9066093BA067093BB06089581
:101D4E00E1E2EA93A091AC06F6CCA091AD0625CDCA
:101D5E00A091AE0627CDA091AF060C944A01E5E105
:101D6E00EA93A091B0060E944A01E2E1E9CCEFE0CD
:101D7E00EA93A091B1060E944A01ECE0EA93A09189
:101D8E00B2060E944A01E9E0EA93A0E20C944A01ED
:101D9E00A091AD060E944A01EBE1D2CCE8E1EA93B4
:101DAE00A091AE060E944A01E5E1EA93D4CFE2E1AA
:101DBE00EA93A091B0060E944A01D9CF0E94251144
:101DCE000E944C10DF01CB010895F0E00E94D71065
:101DDE000E94C70F0E944C100895A091C006B091AA
:101DEE00C1068091C2069091C3060895E091C40683
:101DFE00F091C5066091C6067091C7060895909839
:101E0E009198889A899815C089988898EE2700002D
:101E1E00819B0895809B089504D0899A02D0889A58
:101E2E00E1E061E107C0899A889A03D08898F9DFCA
:101E3E00899861E26A95F1F7089578E08898F1DF64
:101E4E00809BFECFEEDF889481990894889AF1DF0B
:101E5E00EE1F7A9599F77A2F772311F4899801C09E
:101E6E00899ADFDF8898E5DF889ADBDF8998D9CFFA
:101E7E0078E0AA0F10F4899801C0899ADADF889861
:101E8E00D0DF809BFECFCDDF889A7A9591F7899827
:101E9E00C8DF8898CEDFE1E08199EE27889AC1CF1E
:101EAE00109639F084EC99E00197F1F7A895119707
:101EBE00C9F70895552342F4503811F4E0FF04C0D9
:101ECE003196691F791F6BF050E8572711F45F9315
:101EDE00CAC05F3F31F0660F000C57956795752F9E
:101EEE0008955F9300200AF0CAC0C3C050E8192EAF
:101EFE001522880F991F9527550F879550E8072EA5
:101F0E000522660F771F7527550F679508956894FC
:101F1E0001C0E8945F93F2DF703818F07F3F08F449
:101F2E00A2C056E1571BAAF4519558300EF4593001
:101F3E0030F0EFEFFFEF6FEF7FE777F91AC07727FB
:101F4E005523B9F0EE0FFF1F661F771F5A95D1F775
:101F5E0010C07727583028F0EF2FF62F672F5850E4
:101F6E00F9CF552331F076956795F795E7955A9504
:101F7E00D1F700200AF400D15F910895689401C052
:101F8E00E894309760407040B1F0002426F077233B
:101F9E0012F40094F1D0172E7EE1112032F07A95D2
:101FAE00EE0FFF1F661F111CF9CFEF2FF62F612DBD
:101FBE005F938ADF5F9108954F93AF01FD01DA01C0
:101FCE00AB01BC01CA01402D012C142E4F91089576
:101FDE00EA0FFB1F681F0895E095F0956095EF5F7F
:101FEE00FF4F6F4F08955F9381DF903849F150E8AE
:101FFE001526703821F1572F591B2BF112F4DCDF07
:10200E00FACF583118F0AA27BB278827583028F066
:10201E00AB2FB82F88275850F9CF552329F0869526
:10202E00B795A7955A95D9F7502D512572F0D0DF57
:10203E0038F46795F795E795739513F420C0BCDFD8
:10204E0043DF5F910895D8F7FBCFEA1BFB0B680BBC
:10205E0051F010F40094C0DF662392F3EE0FFF1FD1
:10206E00661F7A95CBF7EE27FF27662777275F91B6
:10207E000895EFEFFFEF6FE77FEF5F910895EFEFBA
:10208E00FFEF6FE77FE75F9108955F932FDF703863
:10209E0051F3903841F301240894791F23F41CF373
:1020AE0000203AF3ECCF0F921F932F933F934F9351
:1020BE00112722279927689FA0018F9F302D410D50
:1020CE00591F6B9F300D411D591F8E9F27D0BF9FEB
:1020DE0025D06A9F23D0BE9F1DD0AF9F1BD0AE9F31
:1020EE00110D291F391F491F591FE32FF42F652F7B
:1020FE00522F4F913F912F911F910F9066232AF0EF
:10210E00550FEE1FFF1F661F02C073954BF2D2DEF6
:10211E005F910895100D211D391F02C0200D311D34
:10212E00491F591F089599239AF0772342F0971764
:10213E0048F029F4AE17BF07860720F031F09894C7
:10214E0088940895989408940895189488940895FE
:10215E007723C2F7971798F3A9F7EA17FB076807D3
:10216E0088F399F3ECCFEA2BFB2B682B792B089590
:10217E00F195E195F0400895F09560957095E19593
:10218E00FF4F6F4F7F4F0895EE230E2EFD01BC01C2
:10219E0031F0EE0FFF1F661F771F0A94D1F70895D7
:1021AE006F2F660F660B762F08950024112490E191
:1021BE00AA0FBB1F001C111C0E1A1F0A18F40E0EBC
:1021CE001F1E01C0A1609A9599F7FD01D0010895D7
:1021DE0004D0EBDF0EF4CCDF0895E894F7FF02C0D5
:1021EE00C7DF6894B7FF06C0A095B095119600F8AA
:1021FE00039400FA0895ED91FD916D917D910895EE
:10220E00ED93FD936D937C9308957E936E93FE9361
:10221E00EE930895E881F9816A817B810895A88102
:10222E00B9818A819B810895E883F9836A837B83D0
:10223E0008959A938A93BA93AA930895689401C0C5
:10224E00E89401D09EDE182E862F612D192E972F21
:10225E00712D1B2EBF2FF12D1A2EAE2FE12D0895AD
:00000001FF
